:1000000000308A0068280000FF00030E8301A10071
:100010000A08A0008A010408A2007708A300780853
:10002000A4007908A5007A08A6007B08A70083131E
:1000300083128C308400801E1F288C1A32282208DC
:1000400084002308F7002408F8002508F900260892
:10005000FA002708FB0020088A00210E8300FF0E0B
:100060007F0E09008A110A124D282E308400831356
:10007000000803194C280130F800BF30F700640075
:10008000F70B3F28F80B3D284A30F700F70B4628BE
:1000900000006400800B3B28003483160511831296
:1000A00005150230AD00FA30AE003520AD0B5328F7
:1000B00083160511831205110230AD00FA30AE002F
:1000C0003520AD0B5E284D288C128A110A121F288C
:1000D000840183131F308305333083169900A230C7
:1000E000980090308312980083161F149F141F15D8
:1000F0009F1107309C00FF308312A90083168113E3
:100100001F149F141F159F1183121F1083160912AD
:1001100083129412A91229088316870083122916C4
:100120002908831687008312A911290883168700DE
:100130000130831294000030831694000108C739FF
:1001400008388100831290010030F80092000030DE
:100150008316920007309C00050864000230F70007
:10016000F70BB028B3281C0883120D1383169D01CA
:100170008C16C03083128B04831606148312061863
:10018000EA288316061483120618E92883168511B7
:10019000831285150230AB00A8018B1BA8178B13A7
:1001A000FA30AE003520A81B8B17AB0BCC2883167A
:1001B0008511831285110230AB00A8018B1BA81793
:1001C0008B13FA30AE003520A81B8B17AB0BDD2844
:1001D000C128052964004230F700F70BED280130F3
:1001E000AA062A1CFC2883160512831205168316FC
:1001F00085128312851204298316051283120512B3
:0E0200008316851283128516EA28BC28630037
:02400E00393F38
:00000001FF
